:100000000C942A001895000018950000189500001F
:10001000189500001895000018950000189500002C
:100020001895000018950000189500000C94000326
:10003000189500000C9461120C949312189500000E
:1000400018950000189500001895000018950000FC
:10005000189500008FE58DBFCCEFECE44E2E88E0C4
:100060008EBFD7E0F7E05F2EEEEFF7E0A0E6B0E05E
:10007000A89584B7082E877F84BF88E1992781BD22
:1000800091BD88278D933197E9F788E089B980E0A1
:1000900080BD88E18AB9662484B7877F84BF88E100
:1000A00081BD80E081BD80E08ABB8CE187BB83EEAF
:1000B00088BB80E084BB8FEF85BB80EF81BB8FE086
:1000C00082BB87E886B980E087B9379A85E083BF2D
:1000D00081EB8FBD81E08EBD8FEF8ABD579A0E9464
:1000E0008A13A7E4B1E0EEE1F7E20E94A110A9E4CF
:1000F000B1E0E0E2F7E20E94A110ABE4B1E0E2E29D
:10010000F7E20E94A110AFE4B1E0E6E2F7E20E945C
:10011000A110A3E5B1E0EAE2F7E20E94A110A7E591
:10012000B1E0EEE2F7E20E94A110ABE5B1E0E2E35C
:10013000F7E20E94A110AFE5B1E0E6E3F7E20E942A
:10014000A110A3E6B1E0EAE3F7E20E94A110A7E65E
:10015000B1E0EEE3F7E20E94A110ABE6B1E0E2E429
:10016000F7E20E94A110AFE6B1E0E6E4F7E20E94F8
:10017000A110A3E7B1E0EAE4F7E20E94A110A7E72B
:10018000B1E0EEE4F7E20E94A1108FEF8ABD80E0BB
:1001900088BD00EE14EB27E039E0A0E9B1E00D9353
:1001A0001D932D933C9380E08093C20184E690E000
:1001B000A8EDB1E08D939C93C29A86E990E00E94ED
:1001C0006510C39A86E990E00E946510C49A8AEF90
:1001D00090E00E946510C298C398C49880E090E0B7
:1001E000A6E8B1E08D939C9301E010E020E030E0C0
:1001F000ACE9B1E00D931D932D933C934AE050E0A0
:1002000060E070E0ACE9B1E00D911D912D913C9161
:100210000E94C4121CF011F00C942E01A6E8B1E06B
:100220000D911C910F931F9307B1007E076007B9D2
:100230000E94A710482F592F1F910F91040F151FCF
:10024000A6E8B1E00D931C9381E090E00E94651058
:10025000ACE9B1E00E94110F0C94FE00A6E8B1E0F9
:100260000D911C914AE050E00E94340FA6E8B1E0E5
:100270004D935C9382E090E00E946510A6E8B1E0A7
:100280000D911C91043650E015070CF402C00C943B
:100290004E0184E08093DA010C9491080E949A0A3E
:1002A000789489B7816089BF00913B01013011F0DA
:1002B0000C94880180E080933B01A6EBB0E03FE323
:1002C0000E947D0FA6EBB0E08C91082F0A3011F050
:1002D0000C948601A6EBB0E00E947013082F41E059
:1002E000041BACE3B1E00C93A6EBB0E00E947013EA
:1002F000EA2FFB2F00913C013197E01BF0400FEFFC
:10030000A6EBB0E00E9468130C9462010E94170CE7
:1003100000914601013011F00C9440028BE10E94E3
:10032000CC0FE2E5F7E20E94C20F8BE10E94CC0FF6
:10033000E8E5F7E20E94C20FECE5F7E20E94C20F87
:100340000E94C90FE4E7F7E20E94C20F0E94C90FA2
:10035000ECE8F7E20E94C20FA4E3B7E0E4EAF1E0C0
:100360000E94DA120E94BA0F0E94C90FE8E9F7E270
:100370000E94C20FA4E3B7E0EAEBF1E00E94DA12B8
:100380000E94BA0F0E94C90FE2EAF7E20E94C20F70
:10039000A4E3B7E0E7ECF1E00E94DF120E94BA0F9D
:1003A0000E94C90FEEEAF7E20E94C20FA4E3B7E091
:1003B000E6E8F1E00E94DF120E94BA0F0E94C90F26
:1003C000EEEBF7E20E94C20FA4E3B7E0E4E8F1E04D
:1003D0000E94DF120E94BA0F0E94C90FECECF7E2F4
:1003E0000E94C20FA4E3B7E0E8EAF1E00E94DF1246
:1003F0000E94BA0F0E94C90FECEDF7E20E94C20FF3
:10040000A4E3B7E0EAEAF1E00E94DF120E94BA0F2B
:100410000E94C90FEEEEF7E20E94C20FA4E3B7E01C
:10042000EEEBF1E00E94DA120E94BA0F0E94C90FAF
:10043000E8EFF7E20E94C20FA4E3B7E0EAEDF1E0D3
:100440000E94E6120E94BA0F0E94C90FE4E0F8E28F
:100450000E94C20FA4E3B7E0E2ECF1E00E94E612D2
:100460000E94BA0F0E94C90FEEE0F8E20E94C20F8C
:100470000E94C90F88EC90E00E9465100C94FE0267
:1004800084E190E00E946510E2E1F8E20E94C20F70
:10049000A4E3B7E0E4EAF1E00E94DA120E94BA0FA6
:1004A0000E94C90F84E190E00E946510E8E1F8E243
:1004B0000E94C20FA4E3B7E0EAEBF1E00E94DA1277
:1004C0000E94BA0F0E94C90F84E190E00E9465105B
:1004D000EEE1F8E20E94C20FA4E3B7E0E7ECF1E03E
:1004E0000E94DF120E94BA0F0E94C90F84E190E0BF
:1004F0000E946510E4E2F8E20E94C20FA4E3B7E0B4
:10050000E6E8F1E00E94DF120E94BA0F0E94C90FD4
:1005100084E190E00E946510EAE2F8E20E94C20FD6
:10052000A4E3B7E0E4E8F1E00E94DF120E94BA0F12
:100530000E94C90F84E190E00E946510E0E3F8E2B8
:100540000E94C20FA4E3B7E0E8EAF1E00E94DF12E4
:100550000E94BA0F0E94C90F84E190E00E946510CA
:10056000E6E3F8E20E94C20FA4E3B7E0EAEAF1E0B2
:100570000E94DF120E94BA0F0E94C90F84E190E02E
:100580000E946510ECE3F8E20E94C20FA4E3B7E01A
:10059000EEEBF1E00E94DA120E94BA0F0E94C90F3E
:1005A00084E190E00E946510E2E4F8E20E94C20F4C
:1005B000A4E3B7E0EAEDF1E00E94E6120E94BA0F70
:1005C0000E94C90F84E190E00E946510E8E4F8E21F
:1005D0000E94C20FA4E3B7E0E2ECF1E00E94E61251
:1005E0000E94BA0F0E94C90F84E190E00E9465103A
:1005F000EEE0F8E20E94C20F0E94C90F0C94540171
:100600000F921F922F923F924F925F927F92AF92E2
:10061000BF920F931F932F933F934F935F936F93CB
:100620007F938F939F93AF93BF93CF93DF93EF937A
:10063000FF938FB78F93A89584E6809352000E9412
:10064000CA080E9496040E94CE030E946D050E9473
:1006500045038F918FBFFF91EF91DF91CF91BF91B4
:10066000AF919F918F917F916F915F914F913F914A
:100670002F911F910F91BF90AF907F905F904F90FF
:100680003F902F901F900F901895A8EAB1E00D9120
:100690001C91043B50E015071CF011F00C94520320
:1006A0000C945A0384EB90E0A8EAB1E08D939C93FC
:1006B0000C946B03A8EAB1E00D911C910C345FEF30
:1006C00015070CF402C00C946B038CE49FEFA8EAAE
:1006D000B1E08D939C93AAEAB1E00D911C91043B8B
:1006E00050E015071CF011F00C9478030C94800373
:1006F00084EB90E0AAEAB1E08D939C930C94910373
:10070000AAEAB1E00D911C910C345FEF15070CF4CF
:1007100002C00C9491038CE49FEFAAEAB1E08D93A0
:100720009C93A8EAB1E00D911C91003050E01507B0
:100730000CF402C00C949F03969A0C94A003969814
:10074000AAEAB1E00D911C91003050E015070CF4BD
:1007500002C00C94AE03979A0C94AF039798A8EA42
:10076000B1E08D919C910E94540FA4E9B1E08D936A
:100770009C93AAEAB1E08D919C910E94540FA6E946
:10078000B1E08D939C930FEF40919401041B0ABD3F
:10079000A6E9B1E08C9188BD08950895A4EAB1E07E
:1007A0000D911D912D913C91ACE9B1E00D931D93FC
:1007B0002D933C93ACE9B1E00D911D912D913C91AD
:1007C00041E150E060E070E00E947E10ACE9B1E0F1
:1007D0000D931D932D933D93AAEBB1E00D911D91C7
:1007E0002D913C9141E150E060E070E00E947E106C
:1007F000A8E9B1E00D931D932D933D93A8E9B1E0D5
:100800000D911D912D913C91ACE9B1E04D915D911F
:100810006D917C910E94BA12AEEBB1E00D931D93E5
:100820002D933D93A3ECB1E00D911D912D913C9141
:10083000AEEBB1E04D915D916D917C910E94BA1249
:10084000A3ECB1E00D931D932D933D9348ED56ED30
:1008500060E070E0A3ECB1E00D911D912D913C9111
:100860000E94C4121CF011F00C9438040C94420441
:1008700008ED16ED20E030E0A3ECB1E00D931D9300
:100880002D933C9348E259E26FEF7FEFA3ECB1E088
:100890000D911D912D913C910E94C4120CF402C047
:1008A0000C945C0408E219E22FEF3FEFA3ECB1E0F7
:1008B0000D931D932D933C93A3ECB1E00D911D91ED
:1008C0002D913C914BE950E060E070E00E94FD0FFB
:1008D000ACE9B1E04D935D936D937D93AEEBB1E0E8
:1008E0000D911D912D913C9145EA50E060E070E042
:1008F0000E94FD0FA8E9B1E04D935D936D937D9348
:10090000ACE9B1E00D911D912D913C91A8E9B1E0C8
:100910004D915D916D917C910E94BA12AEEAB1E069
:100920000D931D932D933D930895089500E010E0DD
:1009300020E030E0A8E9B1E00D931D932D933C93A6
:1009400040E050E060E070E0A3ECB1E00D911D915B
:100950002D913C910E94C4121CF011F00C94B20431
:100960000C94C404A3ECB1E00D911D912D913C9128
:1009700040E25EE460E070E00E94BF12A8E9B1E0EE
:100980000D931D932D933D93A8E9B1E00D911D9119
:100990002D913C9146E450E060E070E00E94FD0F34
:1009A000A8E9B1E04D935D936D937D9380E090E075
:1009B000ABEDB1E08D939C934DE050E060E070E0D2
:1009C000A8E9B1E00D911D912D913C910E94C412B6
:1009D0001CF011F00C94EE040C94F8040DE010E0FF
:1009E00020E030E0A8E9B1E00D931D932D933C93F6
:1009F00040E050E060E070E0A8E9B1E00D911D91A9
:100A00002D913C910E94C4120CF402C00C9412056A
:100A100000E010E020E030E0A8E9B1E00D931D9384
:100A20002D933C9340E050E060E070E0A8E9B1E035
:100A30000D911D912D913C910E94C4121CF011F05A
:100A40000C9424050C942A0580E090E0ABEDB1E015
:100A50008D939C9300917B01003011F00C946B05F9
:100A600048EA54EB67E070E0A0E9B1E00D911D9118
:100A70002D913C910E94C4121CF011F00C9442057F
:100A80000C944505C29AC398C49848EA54EB67E0B1
:100A900070E0A0E9B1E00D911D912D913C910E9473
:100AA000C4120CF402C00C945805C39AC498C2989E
:100AB00048E55EE667E070E0A0E9B1E00D911D91C8
:100AC0002D913C910E94C4120CF402C00C946B0551
:100AD000C398C298C49A08950895ACEAB1E00E9400
:100AE000200FACEAB1E00D911C910A3050E01507DF
:100AF0001CF011F00C947E050C948E0500917B0186
:100B0000013011F00C948705C29AC39AC49A0091DF
:100B10007B01023011F00C948E05C49AACEAB1E06E
:100B20000D911C91003150E015071CF011F00C9450
:100B30009B050C94C10500917B01003018F011F069
:100B40000C94A4050C94AC05C298C398C498A9EC65
:100B5000B1E08C918F5F8C9381E090E0ACEAB1E0E2
:100B60008D939C930091C9010A3018F011F00C94F8
:100B7000BB050C94C10580E08093C90180E080939F
:100B80007B01A2EDB1E00D911D9117FB1EF42FEF3B
:100B90003FEF02C022273327A7ECB1E04D915D91D2
:100BA00057FB1EF46FEF7FEF02C0662777270E9486
:100BB000BF12AEECB1E00D931D932D933D93A3ECCA
:100BC000B1E00D911D912D913C9140E25EE460E019
:100BD00070E00E94FD0FA8E9B1E04D935D936D9325
:100BE0007D93A8E9B1E00D911D912D913C910E945A
:100BF0005110A8E9B1E00D931D932D933D9341E071
:100C000050E060E070E0A8E9B1E00D911D912D91F8
:100C10003C910E94C4120CF402C00C94190601E02D
:100C200010E020E030E0A8E9B1E00D931D932D9392
:100C30003C93AEECB1E00D911D912D913C91A8E952
:100C4000B1E04D915D916D917C910E94FD0FAEECF4
:100C5000B1E04D935D936D937D93A3ECB1E00D9165
:100C60001D912D913C9140ED57E060E070E00E94B5
:100C7000FD0FA8E9B1E04D935D936D937D93A8E9D5
:100C8000B1E00D911D912D913C910E945110A8E968
:100C9000B1E00D931D932D933D9346E150E060E04C
:100CA00070E0A8E9B1E00D911D912D913C910E9459
:100CB000C4121CF011F00C945F060C94690606E156
:100CC00010E020E030E0A8E9B1E00D931D932D93F2
:100CD0003C930BE110E020E030E0A8E9B1E04D9159
:100CE0005D916D917C910E94BF12A8E9B1E00D93D6
:100CF0001D932D933D93A8E9B1E00D911D912D9188
:100D00003C914FEF5FEF6FEF7FEF0E947E10A0EA04
:100D1000B1E00D931D932D933D93A8E9B1E04D9162
:100D20005D916D917C91AEECB1E00D911D912D9195
:100D30003C910E94C4121CF011F00C94A1060C947A
:100D4000AD06A8E9B1E00D911D912D913C91AEEC5D
:100D5000B1E00D931D932D933C93A0EAB1E04D912A
:100D60005D916D917C91AEECB1E00D911D912D9155
:100D70003C910E94C4120CF402C00C94CB06A0EA71
:100D8000B1E00D911D912D913C91AEECB1E00D9330
:100D90001D932D933C93AEECB1E00D911D912D91DF
:100DA0003C91A2EBB1E00D931D932D933C93002752
:100DB000A0E3B0E08C9182FB0EF401E040E0041768
:100DC00011F00C94EB068DE790E0A8EDB1E08D9367
:100DD0009C930C940507A8EDB1E00D911C91003394
:100DE00055E715070CF402C00C940207A8EDB1E01A
:100DF0000D911C9141E050E0040F151FA8EDB1E0EA
:100E00000D931C9381E080937B01AEEAB1E00D91DC
:100E10001D912D913C914DE750E060E070E00E9403
:100E20007E10AEEAB1E00D931D932D933D93AEEA93
:100E3000B1E00D911D912D913C91A8EDB1E04D9146
:100E40005D9157FB1EF46FEF7FEF02C06627772797
:100E50000E94FD0FAEEAB1E04D935D936D937D93DB
:100E6000AEEAB1E00D911C91A2EBB1E04D915C9125
:100E7000041B150BA8EAB1E00D931C93AEEAB1E098
:100E80000D911C91A2EBB1E04D915C91040F151FE7
:100E9000AAEAB1E00D931C930091C201003011F059
:100EA0000C94B80780E090E0A8EAB1E08D939C93A1
:100EB00080E090E0AAEAB1E08D939C9300E010E01E
:100EC00020E030E0AEEAB1E00D931D932D933C930A
:100ED00000E010E020E030E0A6EBB1E00D931D93C0
:100EE0002D933C9300E010E020E030E0A3ECB1E073
:100EF0000D931D932D933C9300E010E020E030E033
:100F0000A8E8B1E00D931D932D933C9300E010E011
:100F100020E030E0A4EAB1E00D931D932D933C93C3
:100F200000E010E020E030E0AAECB1E00D931D936A
:100F30002D933C93A6E8B1E00D911C91023350E053
:100F400015071CF011F00C94A7070C94B6070E942B
:100F50009A0A81E08093C20100E010E020E030E0D6
:100F6000AAECB1E00D931D932D933C930C948F0844
:100F7000013011F00C94F807A6E8B1E00D911C9136
:100F8000023350E015070CF402C00C94EC07AAECF5
:100F9000B1E00E94110F40E550E060E070E0AAEC83
:100FA000B1E00D911D912D913C910E94C4121CF055
:100FB00011F00C94DD070C94EA0783E08093C201E2
:100FC00000E010E020E030E0AAECB1E00D931D93CA
:100FD0002D933C930C94F60700E010E020E030E005
:100FE000AAECB1E00D931D932D933C930C948F08C4
:100FF000033011F00C948C0881B5886181BD877F26
:1010000081BD01E010E020E030E0A8E9B1E00D93FF
:101010001D932D933C934FEF50E060E070E0A8E902
:10102000B1E00D911D912D913C910E94C4121CF0D4
:1010300011F00C948408A8EAB1E00D911C910030E5
:1010400050E0150781E009F080E08F93AAEAB1E053
:101050000D911C91003050E0150781E009F080E00F
:101060009F918923882311F40C9438080C948408E8
:10107000A8EAB1E00D911C91003050E015071CF07A
:1010800011F00C9445080C944908A8EAB1E00E94BC
:10109000270FA8EAB1E00D911C91003050E0150730
:1010A0000CF402C00C945808A8EAB1E00E94200F8A
:1010B000AAEAB1E00D911C91003050E015071CF038
:1010C00011F00C9465080C946908AAEAB1E00E943A
:1010D000270FAAEAB1E00D911C91003050E01507EE
:1010E0000CF402C00C947808AAEAB1E00E94200F28
:1010F00089E190E00E9465100E944503A8E9B1E0F3
:101100000E94110F0C940B0880E08093C20181B5FE
:10111000886081BD0C948F0883E08093C20108959C
:10112000089581B5886181BD877F81BD01E010E0B0
:1011300020E030E0ACE9B1E00D931D932D933C939A
:10114000AAEDB1E04C91552766277727ACE9B1E0CD
:101150000D911D912D913C910E94C4121CF011F033
:101160000C94C208C49A86E990E00E946510C49865
:1011700086E990E00E946510ACE9B1E00E94110F91
:101180000C94A008E2E0F0E00E94F40F0C949608A2
:101190000895089507B1007E056007B90E94A71061
:1011A000A0E8B1E08D939D9388278D938C9300E008
:1011B00014E020E030E0A0E8B1E04D915D916D9148
:1011C0007C910E94BF12A0E8B1E00D931D932D9376
:1011D0003D9307B1007E036007B90E94A710ACE7FA
:1011E000B1E08D939D9388278D938C9307B1007EFA
:1011F000006007B90E94A710A4E8B1E08D939C930A
:1012000007B1007E066007B90E94A710A7ECB1E005
:101210008D939C9300E014E00F931F9307B1007E21
:10122000076007B90E94A710482F592F1F910F91EF
:10123000041B150BA6E8B1E00D931C93A8E8B1E0E0
:101240000D911D912D913C914CE251E060E070E0D8
:101250000E94FD0FACE9B1E04D935D936D937D93DA
:10126000A8E8B1E00D911D912D913C91ACE9B1E060
:101270004D915D916D917C910E94BF12A8E8B1E003
:101280000D931D932D933D93ACE7B1E00D911D910E
:101290002D913C91A4EDB1E04D915C9166277727AB
:1012A0000E94BF12ACE9B1E00D931D932D933D93C5
:1012B000ACE9B1E00D911D912D913C91ABEDB1E008
:1012C0004D915D9157FB1EF46FEF7FEF02C06627D3
:1012D00077270E94BA12ACE9B1E00D931D932D93CC
:1012E0003D93A8E8B1E00D911D912D913C91ACE9A1
:1012F000B1E04D915D916D917C910E94BA12A8E888
:10130000B1E00D931D932D933D93ACE8B1E00D91A9
:101310001D912D913C914CE251E060E070E00E9403
:10132000FD0FA8E9B1E04D935D936D937D93ACE81B
:10133000B1E00D911D912D913C91A8E9B1E04D9145
:101340005D916D917C910E94BF12ACE8B1E00D936C
:101350001D932D933D93ACE8B1E00D911D912D911E
:101360003C91A0E8B1E04D915D916D917C910E941E
:10137000BA12ACE8B1E00D931D932D933D93ACE808
:10138000B1E00D911D912D913C914EE150E060E056
:1013900070E00E94FD0FA8E9B1E04D935D936D935D
:1013A0007D93A0E8B1E00D911D912D913C914AE013
:1013B00050E060E070E00E947E10ACE9B1E00D9377
:1013C0001D932D933D93A8E9B1E00D911D912D91B1
:1013D0003C91ACE9B1E04D915D916D917C910E94A1
:1013E000BF12A8E9B1E00D931D932D933D93A8E999
:1013F000B1E00D911D912D913C9143E250E060E0F0
:1014000070E00E947E10A8E9B1E00D931D932D932A
:101410003D93A8E9B1E00D911D912D913C9144E6D9
:1014200050E060E070E00E94FD0FA8E9B1E04D934C
:101430005D936D937D93A8E9B1E00D911D912D9180
:101440003C91AAEBB1E00D931D932D933C93AAEB35
:10145000B1E00D911D912D913C91A8E9B1E00D9362
:101460001D932D933C93A8E8B1E00D911D912D9112
:101470003C91A8E9B1E04D915D916D917C910E9404
:10148000BA12A8E8B1E00D931D932D933D93A8E8FF
:10149000B1E00D911D912D913C914EE150E060E045
:1014A00070E00E94FD0FA4EAB1E04D935D936D934F
:1014B0007D93A0E9B1E00D911D912D913C914CE2FD
:1014C00051E060E070E00E94FD0FA8E9B1E04D93AB
:1014D0005D936D937D93A0E9B1E00D911D912D91E8
:1014E0003C91A8E9B1E04D915D916D917C910E9494
:1014F000BF12A0E9B1E00D931D932D933D93A0E998
:10150000B1E00D911D912D913C91A4E8B1E04D9178
:101510005D9157FB1EF46FEF7FEF02C066277727C0
:101520000E94BA12A0E9B1E00D931D932D933D9353
:101530000895089581B5886181BD877F81BD80E070
:1015400090E0A7ECB1E08D939C9301E010E020E0E7
:1015500030E0ACE9B1E00D931D932D933C934AE04C
:1015600050E060E070E0ACE9B1E00D911D912D918B
:101570003C910E94C4121CF011F00C94DF0AA7ECFD
:10158000B1E00D911C910F931F9307B1007E06608F
:1015900007B90E94A710482F592F1F910F91040FD0
:1015A000151FA7ECB1E00D931C9381E090E00E9421
:1015B0006510ACE9B1E00E94110F0C94AF0AA7ECE2
:1015C000B1E00D911C914AE050E00E94340FA2ED71
:1015D000B1E04D935C9300E010E020E030E0A0E843
:1015E000B1E00D931D932D933C9301E010E020E0BA
:1015F00030E0ACE9B1E00D931D932D933C9344E6AC
:1016000050E060E070E0ACE9B1E00D911D912D91EA
:101610003C910E94C4121CF011F00C944C0B07B1C9
:10162000007E056007B90E94A710A8E9B1E08D937C
:101630009D9388278D938C9300E014E020E030E0A8
:10164000A8E9B1E04D915D916D917C910E94BF122E
:10165000A8E9B1E00D931D932D933D93A0E8B1E06F
:101660000D911D912D913C91A8E9B1E04D915D91B5
:101670006D917C910E94BA12A0E8B1E00D931D9388
:101680002D933D9382E090E00E946510ACE9B1E0BB
:101690000E94110F0C94FF0AA0E8B1E00D911C917B
:1016A00044E650E00E945A0FA6EDB1E04D935C93E2
:1016B0000CE211E020E030E0A6EDB1E04D915C914C
:1016C000662777270E947E10ACE8B1E00D931D934A
:1016D0002D933D9300E010E020E030E0ACE7B1E076
:1016E0000D931D932D933C9301E010E020E030E03A
:1016F000ACE9B1E00D931D932D933C9344E650E08B
:1017000060E070E0ACE9B1E00D911D912D913C914C
:101710000E94C4121CF011F00C94B90B07B1007EAA
:10172000036007B90E94A710A8E9B1E08D939D93CB
:1017300088278D938C93ACE7B1E00D911D912D918D
:101740003C91A8E9B1E04D915D916D917C910E9431
:10175000BA12ACE7B1E00D931D932D933D9382E057
:1017600090E00E946510ACE9B1E00E94110F0C946A
:101770007E0BACE7B1E00D911C9144E650E00E9475
:101780005A0FA4EDB1E04D935C9381B5886081BDA3
:10179000A4EDB1E00D911C91003951E0150710F056
:1017A0000C94D70B83E08093DA010C949108A4ED9C
:1017B000B1E00D911C91083552E0150718F011F0B9
:1017C0000C94E40B0C94E90B83E08093DA010C9405
:1017D0009108A6EDB1E00D911C910E3551E0150771
:1017E00010F00C94F80B82E08093DA010C949108CD
:1017F000A6EDB1E00D911C910E3E52E0150718F0D8
:1018000011F00C94050C0C940A0C82E08093DA0120
:101810000C9491080895089581E080933B01089508
:10182000A6EBB0E00E94BC0F0E94C90F0895A6EB82
:10183000B0E08C91082F033211F00C94230C0E941D
:10184000100C0C94A00CA6EBB0E08C91082F0B317F
:1018500011F00C942F0C0E94100C0C94A00CA6EB11
:10186000B0E0EEE1F7E22FEF91E00E94B510A5E4C1
:10187000B1E00C9300914501003018F011F00C9488
:10188000430C0C94900CA6EBB0E0EEE4F8E22FEFE2
:1018900091E00E94B510002F003080E010F009F0B8
:1018A00081E08F9340914501A6EBB0E0EEE4F8E2D1
:1018B0002FEF91E00E94B510002F041781E008F08F
:1018C00080E09F918923882311F40C946F0C0E946F
:1018D000100C0E94A10C0C94A00C0C948E0CE6EB46
:1018E000F0E000914501A6EFB0E00E946813A6EF7A
:1018F000B0E00E943013ADE3B1E00C9300913D01E4
:10190000003011F00C948A0C0E94A10C0C94A00CD5
:101910000C948E0C0E94100C0C94A00C0C94A00C37
:1019200000913D01003011F00C949C0C0E94A10C20
:101930000C94A00C0C94A00C0E94100C0C94A00C05
:10194000089581E08093DE01A6EFB0E088278C93B4
:10195000A6E3B1E088278C93A0E4B1E0EAE1F7E2E6
:101960000E944D1280E090E0AEE3B1E08D939C9335
:10197000A6EBB0E00E947013082F0F93A6EBB0E027
:10198000E7E4F1E0222791E00E94B510402F0F918B
:10199000041BA5E4B1E00C93A6EBB0E00E94701329
:1019A000EA2FFB2F009145013197E01BF0400FEF2C
:1019B000A6EFB0E00E94681381E08093DD01009102
:1019C000DD01043018F011F00C945A0D81E4482F19
:1019D000ADEDB1E0AD90BB24A5EFB0E0AA0DBB1D0D
:1019E0000C91041781E008F480E08F938AE5482F7A
:1019F000ADEDB1E0AD90BB24A5EFB0E0AA0DBB1DED
:101A00000C91041781E010F009F080E09F91892388
:101A10008F9381E6482FADEDB1E0AD90BB24A5EFEB
:101A2000B0E0AA0DBB1D0C91041781E008F480E022
:101A30009F91892B8F938AE7482FADEDB1E0AD9050
:101A4000BB24A5EFB0E0AA0DBB1D0C91041781E0EB
:101A500010F009F080E09F918923882311F40C9401
:101A6000520DADEDB1E0AD90BB24A5EFB0E0AA0DF5
:101A7000BB1D8C91AEEDB1E0AD90BB24A5E3B1E010
:101A8000AA0DBB1D8C93AEEDB1E08C918F5F8C9352
:101A900080E0AEEDB1E0AD90BB24A5E3B1E0AA0DCE
:101AA000BB1D8C93ADEDB1E08C918F5F8C9310F4E6
:101AB0000C94DF0CA6E3B1E00E947013082F0330F2
:101AC00011F00C94980DE6E3F1E0A6E3B1E00E947A
:101AD000551280E08093DD010091DD01093118F09D
:101AE00011F00C94980DEDEDF1E00191112744E017
:101AF00050E00E947410E7E4F1E0E00FF11FA6E36C
:101B0000B1E00E94781311F00C94900DADEDB1E0AE
:101B10008C91AEE3B1E08D9388278C930C94980D53
:101B2000ADEDB1E08C918F5F8C9310F40C946C0D43
:101B300081E08093DE01A6E3B1E088278C93A6EFD5
:101B4000B0E0E9E4F1E0222791E00E94B510A5E4BD
:101B5000B1E00C9300914501003011F00C94B70DE9
:101B6000A6EFB0E00E947013A5E4B1E08C9381E091
:101B70008093DD01409145010091DD01041718F0CB
:101B800011F00C94120E80E3482FADEDB1E0AD9052
:101B9000BB24A5EFB0E0AA0DBB1D0C91041781E09A
:101BA00008F480E08F9389E3482FADEDB1E0AD906C
:101BB000BB24A5EFB0E0AA0DBB1D0C91041781E07A
:101BC00010F009F080E09F918923882311F40C9490
:101BD0000A0EADEDB1E0AD90BB24A5EFB0E0AA0DCB
:101BE000BB1D8C91AEEDB1E0AD90BB24A5E3B1E09F
:101BF000AA0DBB1D8C93AEEDB1E08C918F5F8C93E1
:101C000080E0AEEDB1E0AD90BB24A5E3B1E0AA0D5C
:101C1000BB1D8C93ADEDB1E08C918F5F8C9310F474
:101C20000C94BA0DAEE3B1E00D911C910F931F938C
:101C3000A6E3B1E00E943013402F512F1F910F9166
:101C4000040F151FAEE3B1E00D931C93A6EFB0E0B7
:101C5000E9E4F1E0222791E00E94B510002F003066
:101C600018F011F00C94360E0C943D0E8091440146
:101C70008F77809344010C94420E809144018068D8
:101C800080934401A6EFB0E00E947013082F0F93D9
:101C9000A6EFB0E0E9E4F1E0222791E00E94B51060
:101CA000402F0F91041BA5E4B1E00C93A6EFB0E028
:101CB0000E947013EA2FFB2F009145013197E01B22
:101CC000F0400FEFA6EFB0E00E946813A6EFB0E07F
:101CD0000E947911EDE0F0E0A0E4B1E00E9462130F
:101CE000AEE3B1E00D911C91013050E0150711F009
:101CF0000C94940EA6EBB0E0E0E5F8E20E94A1108F
:101D0000A6EBB0E00E94740FECE7F1E00E94DA125B
:101D1000A6EBB0E00E94740FE8E5F8E20E94A11083
:101D20000E94100C0C94100F023050E0150711F0B7
:101D30000C94B40EA6EBB0E0EAE5F8E20E94A11024
:101D4000A6EBB0E00E94740FE0E8F1E00E94DA1226
:101D5000A6EBB0E00E94740FE8E5F8E20E94A11043
:101D60000E94100C0C94100F033050E0150711F076
:101D70000C94C40EA6EBB0E0E2E6F8E20E94A110DB
:101D80000E94100C0C94100F043050E0150711F055
:101D90000C94DD0E81E0809346018BE10E94CC0F14
:101DA000E2E5F7E20E94C20F8BE10E94CC0FE8E56A
:101DB000F7E20E94C20F0C94100F053050E0150797
:101DC00011F00C94E80E80E0809346010C94100F03
:101DD000063050E0150711F00C94080FA6EBB0E0A8
:101DE000EEE8F8E20E94A110A6EBB0E00E94740FAA
:101DF000E4E8F1E00E94DF12A6EBB0E00E94740F6D
:101E0000E8E5F8E20E94A1100E94100C0C94100F5B
:101E1000A6EBB0E0E6E9F8E20E94A1100E94100CE7
:101E200008950D911D912D913C9181E0080F882717
:101E3000181F281F381F3C932E931E930E9308954E
:101E4000ED91FC91EF5FFF4FFC93EE930895ED91C0
:101E5000FC91E150F040FC93EE93089509D00E946C
:101E6000741000FC10D0089503D024D001F8F9CFED
:101E70000024E89457FF02C009D0689400F80BD002
:101E800010F80124089502D009D008955095409586
:101E90004F5F5F4F0895E89417FF089500951095E0
:101EA0000F5F1F4F6894089599231AF480959095B9
:101EB00001960895352F242FE894452B11F468944A
:101EC0000895512F402F0027112780E1440F551FFF
:101ED000001F111F021B130B416018F4020F131F88
:101EE0004E7F8A9599F708958F938D918823E9F70E
:101EF00011978F910895A4E3B7E018D0883091F03E
:101F00008D3039F03323C9F38D933A9563FE44D075
:101F1000F4CF63FC04C08DE03FD08AE03DD0882739
:101F20008C93089539D011973395E7CF0F929F93F3
:101F3000AF93BF937F9380918A008823E1F3F89455
:101F400080918A008A9580938A0090918800A0E60B
:101F5000B0E0A90F0024B01D8C919395983209F43C
:101F600099279093880078947F91BF91AF919F912A
:101F70000F900895A4E3B7E08D91882311F00CD061
:101F8000FBCF08950E947511802D11F005D0FACF76
:101F900008958DE001D08AE09F939FB79F93AF9300
:101FA000BF930F937F939091B5009832E1F3F8942B
:101FB0009091B50093959093B50099270091B40046
:101FC000ABE8B0E0A00FB91F8C930395083209F479
:101FD00000270093B400559A7F910F91BF91AF9164
:101FE0009F919FBF9F91089588EE93E06ED03197A7
:101FF000D9F7089500FC05D0089530D005D001F838
:10200000F9CF37D03FD00895842F952FA62FB72F23
:10201000E894452B462B472B11F468940895402FE4
:10202000512F622F732F0027112722273327F0E229
:10203000440F551F661F771F001F111F221F331FDC
:10204000081B190B2A0B3B0B416028F4080F191FC2
:102050002A1F3B1F4E7FFA9559F708950024E894F4
:1020600077FF02C006D0689400F809D010F8012468
:10207000089512D04F5F5F4F6F4F7F4F0895E894E0
:1020800037FF089500951095209530950F5F1F4FED
:102090002F4F3F4F689408954095509560957095E7
:1020A000089537FF089500951095209530950F5F9E
:1020B0001F4F2F4F3F4F08953197F1F708956894C0
:1020C00062F80895E89462F80895EF93FF93EE277D
:1020D000E82BE92B31F0E0EAFFE03197F1F70197C7
:1020E000D1F7FF91EF9108950F92B801469F8001BB
:1020F000479F100D569F100D0F9008950F921F923D
:102100002F92C801D901489F80014A9F90014B9F9F
:10211000202C499F100D211D321D5A9F202C589FA5
:10212000100D211D321D599F200D311D689F200D5E
:10213000311D699F300D789F300D2F901F900F90AB
:1021400008950E9475110D920020D9F70895369ACE
:102150003699FECF369A3699FECF84B195B108955F
:1021600099910027A90FB01F1197492F4A955E2F0B
:102170006F2FE89411274395203019F0C895802DD2
:1021800001C080818823B9F07C917723A1F0781772
:1021900039F40EF0042F1395689411963196EBCF15
:1021A000112321F0411BA11B1127B10BE894E52F4E
:1021B000F62F1196E0CF882311F000270895089597
:1021C000D190E190F1900191089521913191419147
:1021D00051910895102F90E8FF0C001F0927990FC7
:1021E000F7941078652F90E8440F551F5927990FE1
:1021F0004795607800380895FF0C90E89027110FFC
:102200009795F794092F0895502F2D2D3E2D4F2D82
:10221000612F08952DEC3CEC4CEC5DE366270FC07C
:10222000CFDFF2DFDD24EE2490E8F92E0FE307C0C4
:10223000CCDF05C02227332740E251E4662755232F
:1022400051F1002381F1C6DF71F116270058505873
:102250000894050B18F407FD03C025C007FD23C033
:10226000469537952795F694E794D79422D0FF208A
:102270002AF0DD0CEE1CFF1C015073F09D2D96958D
:1022800048F0DD203AF4EE202AF491E0D90E9927A7
:10229000E91EF91EB1CF07C09FE7092FF92A9FEF6A
:1022A000D92EE92E0895DD24EE24FF2400271127DE
:1022B00008959F929924AA24BB2488E1D216E306AC
:1022C000F40628F0D21AE30AF40A089401C08894AC
:1022D000991CAA1CBB1CDD0CEE1CFF1C8A9571F717
:1022E000D92CEA2CFB2C9F900895C895319600209C
:1022F00008950E946210E89488278A938A93D3DF16
:1023000011278D918032E9F31197BBD098F08D326F
:1023100029F4109511968C91B4D060F08E3229F486
:1023200011968C91AED008F446C022960E945F10A0
:1023300081E008958C91A5D0D8F547D01196D0F7BB
:1023400003958D919ED0E0F38E3229F48C9199D033
:1023500010F41196FBCF853419F0853609F055C07D
:1023600011968C918ED060F08D3219F08B3221F065
:10237000DCCF08800094088211968C9182D0A8F658
:102380008053898311968C917CD058F49981990F50
:10239000990F0980900D990F8053890F8983873297
:1023A00020F68981988199230AF48195080F2DC020
:1023B0008E3289F611968C9164D068F606D018F0AA
:1023C00011960A95F8CF1196C1CF4F2D3E2D2D2D88
:1023D000DD0CEE1CFF1CA8F0DD0CEE1CFF1C88F0D1
:1023E000D20EE31EF41E68F0DD0CEE1CFF1C48F05C
:1023F000805309F06894D80E8827E81EF81E08F06C
:102400000895F42EE32ED22E089534D019F116F546
:10241000098308E921D00695882787959F2D9F7706
:10242000980FF92E0150000F110F0795898188230D
:1024300079F01AF48195898306C0ECDE89818A954A
:102440008983D9F705C0F6DE89818A958983D9F712
:102450002296089528DFFCCF0DD041F0FF2032F006
:102460000A9531F0DD0CEE1CFF1CD2F7889408951C
:102470000894089500240D280E280F28002A002013
:102480000895803320F08A3310F4089408958894D6
:10249000089591E005C092E003C094E001C098E087
:1024A00024DF0D929A95E1F70895819104D08D93E0
:1024B0008823D9F70895813618F08B3708F48F7D7B
:1024C00008957F930F93AF93BF938F939F938FB78D
:1024D0008F93E89480918A0008E2081B21F49CB154
:1024E0000E945F1013C000918900A0E6B0E077273A
:1024F0009CB1A00FB71F9C936894839580938A002A
:102500000395083209F40027009389009D3011F4E7
:102510000E940C0C8F918FBF9F918F91BF91AF91B3
:102520000F917F9118957F93AF93BF938F939F9354
:102530008FB78F939091B500992399F09A959093C6
:10254000B5009927ABE8B0E08091B300A80FB91FA0
:102550009C918395883209F488278093B3009CB9B5
:1025600001C055988F918FBF9F918F91BF91AF916F
:102570007F911895040F151F261F371F0895041B00
:10258000150B260B370B0895041715072607370779
:102590000895000F111F221F331F089500951095F5
:1025A000209530950F5F1F4F2F4F3F4F089501919A
:1025B00010810EC001911191219130810BC00191C8
:1025C000108117FF05C03FEF2FEF04C000811127D6
:1025D0002227332737FF03C0E1DF8DE28D93CF93AE
:1025E000DF93CF92DF92EF92AA24BB24CC24DD2488
:1025F000EE2440E2CAE0DD2755E093E38881890FAD
:1026000087FD9F7083FD907F891B89935A95A9F759
:10261000C0DFAA1CBB1CCC1CDD1CEE1C4A9551F76C
:10262000E894EFE0FF2782910ED0EB30E0F71EF048
:1026300068948A2D0CD088278D93EF90DF90CF90EF
:10264000DF91CF910895982F829501D0892F8F70B7
:10265000805D26F0803309F4089568948D93089581
:1026600000271127222733271DD08A3328F48033EF
:1026700018F005D015D0F9CF0EF490CF08958053FF
:102680008F93402F512F622F732F83DF82DF72DFF2
:1026900080DF8F919927080F191F291F391F08956F
:1026A0008D910895E894FCDF8032E9F38B32D9F301
:1026B0008930C9F38D3211F46894F2CF08958827D8
:1026C0008D93089594E081918D939A95E1F7089503
:1026D00081918D930A9519F08823D1F70895EFCF52
:1026E0008FEF83959D919923E1F70895689401C038
:1026F000E894AF93BF938D9116F0919103C00E941F
:102700007511902D891718F011F48823A1F7BF9146
:10271000AF910895689463F80895000000003A00AE
:102720003D00414458004944470049444E00544547
:102730004C005354500053574900424154004D4FF0
:1027400041004D4F420053545200455252004D4FEC
:1027500044005B313B3166005B324A002354656CB8
:10276000656D65747269652076312E3020202020D9
:102770002020000023202020202020202020202096
:10278000202020202020202020200000234E6569CA
:1027900067756E67203D2000234779726F203D20CA
:1027A0000000234C656E6B6572203D2000002346BF
:1027B00075DF736368616C746572203D200023428D
:1027C00061747465726965203D200000234D6F744B
:1027D0006F72206C696E6B73203D2000234D6F7407
:1027E0006F7220726563687473203D20000023536C
:1027F000747265DF203D2000234665686C65722099
:102800003D200000234D6F647573203D2000313A58
:102810003400323A313D0000323A333D0000323A62
:10282000353D0000323A363D0000323A373D000077
:10283000323A383D0000323A393D0000323A313008
:102840003D00323A31313D00323A31323D002A000A
:1028500023303A4144583D00210023303A4944474F
:102860003D0023303A49444E3D5B4350552D4D6F5A
:1028700064756C2076332E3320626574612047FCCA
:102880006E746572204765726F6C645D2100233041
:102890003A4241543D0023303A4552523D5B537910
:0E28A0006E746178204572726F725D210000C7
:00000001FF
